:1000000012C043C01895189518951895189518950D
:100010001895189518951895189518951895189578
:100020001895189518958FED8DBFC0ECE0EC4E2E0D
:10003000DD275D2EEEE7F0E0A0E6B0E088278D93A7
:100040003197E9F766248FE087BB8BEF81BB80E7B0
:1000500088BB84E082BB939A84E690E08ED3939829
:1000600084E690E08AD3939A84E690E086D39398CE
:1000700078948BB780648BBFC398C298C198C0989E
:1000800085B7806385BF8895F7CFEAE0F0E0AEE6FC
:1000900091E0ADD300916E000E3C08F004C085B72E
:1000A000806385BF8895E3E1F0E0AEE691E09FD301
:1000B00000916E000E3C08F004C085B7806385BFD8
:1000C000889500916F00043610F009F001C004C05B
:1000D00085B7806385BF8895C39AC29AC19AC09A32
:1000E00080E080936A0080E080936900ACE654D39E
:1000F000A1E654D380E080936500ACE6E2D2C39AD7
:10010000C0988CE080936000BC98A0E79C9197FF1A
:1001100004C0B49B0EC09F779C93B4990AC088E238
:100120009F9399272AD39F91B49903C090689C9379
:1001300032D18AE080936000BD98A0E79C9196FF41
:1001400004C0B59B0EC09F7B9C93B5990AC088E202
:100150009F93992712D39F91B59903C090649C9364
:100160001AD18BE080936000BE98A0E79C9195FF28
:1001700004C0B69B0EC09F7D9C93B6990AC088E2CE
:100180009F939927FAD29F91B69903C090629C934E
:1001900002D1C09AC19889E080936000BC98A0E722
:1001A0009C9197FF04C0B49B0EC09F779C93B49919
:1001B0000AC088E29F939927E0D29F91B49903C027
:1001C00090689C93E8D088E080936000BD98A0E799
:1001D0009C9196FF04C0B59B0EC09F7B9C93B599E4
:1001E0000AC088E29F939927C8D29F91B59903C00E
:1001F00090649C93D0D087E080936000BE98A0E785
:100200009C9195FF04C0B69B0EC09F7D9C93B699B0
:100210000AC088E29F939927B0D29F91B69903C0F4
:1002200090629C93B8D0C19AC29886E08093600097
:10023000BC98A0E79C9197FF04C0B49B0EC09F7729
:100240009C93B4990AC088E29F93992796D29F9174
:10025000B49903C090689C939ED085E08093600021
:10026000BD98A0E79C9196FF04C0B59B0EC09F7BF4
:100270009C93B5990AC088E29F9399277ED29F915B
:10028000B59903C090649C9386D084E0809360000D
:10029000BE98A0E79C9195FF04C0B69B0EC09F7DC1
:1002A0009C93B6990AC088E29F93992766D29F9142
:1002B000B69903C090629C936ED0C29AC39883E0B3
:1002C00080936000BC98A0E79C9197FF04C0B49B0A
:1002D0000EC09F779C93B4990AC088E29F93992798
:1002E0004CD29F91B49903C090689C9354D082E003
:1002F00080936000BD98A0E79C9196FF04C0B59BD9
:100300000EC09F7B9C93B5990AC088E29F93992762
:1003100034D29F91B59903C090649C933CD081E006
:1003200080936000BE98A0E79C9195FF04C0B69BA7
:100330000EC09F7D9C93B6990AC088E29F9399272F
:100340001CD29F91B69903C090629C9324D0BF9811
:10035000A0E79C9194FF04C0B7990EC09F7E9C9328
:10036000B79B0AC088E29F93992707D29F91B79BBA
:1003700003C090619C9392D181E090E0FED1ACE605
:100380000D911C91083853E1150710F009F001C0D8
:10039000B4CE18950895ACE6FFD1939A84E690E028
:1003A000ECD1939884E690E0E8D1A6E30C9104FBAD
:1003B00081E00EF480E08F93A6E30C9105FB81E0D1
:1003C0000EF480E09F91892B8F93A6E30C9106FB9E
:1003D00081E00EF480E09F91892B882309F401C00D
:1003E000E4CF00916900013009F015C080916000F0
:1003F00080936A0000916A00033010F009F001C098
:1004000001C0CEC0A9E68C918F5F8C9380E0809371
:100410006500F8D0089500916900023009F001C02C
:1004200047C000916900033009F001C060C000912D
:1004300060000B3009F008C0A9E68C918F5F8C93A7
:1004400080E0809365000895009160000C3009F011
:100450002EC048EE53E060E070E0A1E60D911D91E2
:100460002D913C91A6D10CF401C002C099C01FC0CF
:10047000E2E0F0E0A4E194E0BAD19BD109F002C03F
:10048000E5C015C0E6E0F0E0A4E194E0B0D191D180
:1004900009F002C0DBC00BC0EBE0F0E0A4E194E0A7
:1004A000A6D187D109F002C0D1C001C079C04CC02B
:1004B000009160000C3009F019C0E2E0F0E0A4E126
:1004C00094E095D1A1E60D911D912D913C9171D1B2
:1004D00009F401C065C096D0A1E660D180E08093A8
:1004E0006500A9E68C918F5F8C9308952DC00091D3
:1004F00060000C3009F028C000916A00013009F05A
:1005000007C0E2E0F0E0A1E694E07BE75FD115C030
:10051000023009F007C0E6E0F0E0A1E694E07BE7F6
:1005200055D10BC0033009F007C0EBE0F0E0A1E6C5
:1005300094E07BE74BD101C033C064D08CEE93E1F3
:10054000ACE68D939C930895A5E68C918F5F8C9378
:1005500000916500063010F009F001C001C020C014
:10056000A1E60D911D912D913C914AE050E060E093
:1005700070E0B4D0A1E60D931D932D933D93A1E6B9
:100580000D911D912D913C91A0E64C915527662728
:1005900077270AD1A1E60D931D932D933D930895DE
:1005A000ABE68C918F5F8C93AFE68C918F5F8C93D1
:1005B00089E0809367008FE5809368002BD00091DD
:1005C0006B00033009F018C0ECE3F0E081D080E06C
:1005D00080936B0080916E00815080936E00EAE002
:1005E000F0E0AEE691E07BE7F1D0E3E1F0E0AEE6EB
:1005F00091E07BE7EBD006D08CEE93E1ACE68D93F7
:100600009C93089582E08093670088EC8093680053
:1006100001D0089581E080936600409167000091C9
:100620006600041710F009F010C0939AA8E68C91A8
:100630009927A3D09398A8E68C9199279ED0A6E6F7
:100640008C918F5F8C9308F4E8CF089580E08093BD
:100650006B00A1E6A3D0D6DF84EF91E08ED0949A10
:10066000E1E0F0E035D09498E1E0F0E031D0809125
:100670006E00815080936E00EAE0F0E0AEE691E01B
:100680007BE7A4D0E3E1F0E0AEE691E07BE79ED02B
:100690008CEE93E1ACE68D939C930895E4E0F0E05A
:1006A00017D0B79901C00CC0E2E0F0E002ED14E011
:1006B00020E030E0A0E1BB2794E07BE787D0A2DF19
:1006C0000895ED91FC91EF5FFF4FFC93EE93089539
:1006D00088EE93E052D03197D9F7089522D006D012
:1006E00000FC01D0089528D030D00895842F952F94
:1006F000A62FB72F4427552766277727F1E288943E
:1007000009C020F4480F591F6A1F7B1F7695679513
:10071000579547953795279517950795FA9589F732
:1007200008950024E89477FF02C006D0689400F88A
:1007300009D010F80124089512D04F5F5F4F6F4F1A
:100740007F4F0895E89437FF089500951095209500
:1007500030950F5F1F4F2F4F3F4F6894089540957E
:1007600050956095709508953197F1F708956894C4
:1007700062F80895E89462F80895EF93FF93EE27E6
:10078000E82BE92B31F0EAEFF0E03197F1F7019730
:10079000D1F7FF91EF91089582E001C084E099279D
:1007A0009D938A95E9F70895040F151F261F371F9B
:1007B000089504171507260737070895E199FECF16
:1007C000EEBB3196089591E001C092E07B3751F481
:1007D0007FB7F894F3DF8D918DBBE29AE19A9A95F9
:1007E000C9F77FBF7727089591E001C092E0E6DF67
:0C07F000E09A8DB38D939A95D1F708958F
:00000001FF
